:100000008031252B0000203085001C308400000842
:10001000031917280230F800F701F70B0D28F80B29
:100020000C289730F700F70B1328800B0A280800DC
:10003000FF3021008C008D0022008D1021008D10DA
:1000400022000D1021000D1024008D0021009513B9
:1000500022000C1221000C120D168D158D178D1615
:100060000D170D158C178C1522008C1521000C1105
:1000700022000C1521001E129E161E139E171D1421
:100080001E109E101E11013023008C0000308D00C8
:10009000F80021001D08C33978049D002000A2014A
:1000A000A101A3018031432B22000C1557285828A9
:1000B0008C1121008C115C285D2822000C11602815
:1000C00061282000080021008C156628672822007E
:1000D0000C156A286B280C116D286E28200008006A
:1000E00022008C1121008C117528762822000C1515
:1000F00079287A280C117C287D2820000800BB0173
:100100003B08063C031C8D28BA1F882863208928D9
:1001100070200310BA0DBB0A80280800BA01210024
:100120008C159228932822000C15962897282000D9
:100130008C1DA2289B289C28BA0A3A08643C031903
:10014000A228982822000C11A528A628A728A828AC
:100150008C1121008C11AC28AD2820003A08643C99
:10016000031DBD280430BB00FA30BC000320BB0BCC
:10017000B4280130F800C028C0280030F800C0289A
:10018000080022008C1121008C11C628C7282200EB
:100190000C15CA28CB2821008C15CE28CF2820008A
:1001A000080054203608BA007F2070208E20F808FE
:1001B0000319DE28C1200130F8000D29B9013908E2
:1001C000073C031CEC28B71FE7286320E8287020B1
:1001D0000310B70DB90ADF288E20F8080319F42898
:1001E000C1200130F8000D29B9013908073C031C72
:1001F0000229B81FFD286320FE2870200310B80DC7
:10020000B90AF5288E20F80803190A29C1200130FF
:10021000F8000D29C1200030F80008003308023C26
:10022000031D2929F530B40534080A38B5002030FB
:10023000B6003308B7003508B800D12034080838B4
:10024000B5002230B6003308B7003508B800D12019
:1002500037292030B6003308B7003408B800D12061
:100260002230B6003308B7003408B800D1200800A7
:1002700054203308BA007F2070208E20F80803191C
:100280004529C1200130F800A829B5013508073CEF
:10029000031C5329B41F4E2963204F2970200310DB
:1002A000B40DB50A462922000C15562957292100FC
:1002B0008C155A295B2922000C115E295F290C1527
:1002C000612962298C1121008C116629672922007D
:1002D0000C116A296B2920003308BA007F206320A3
:1002E0008E20F80803197829C1200130F800A829C8
:1002F000B601B5013508073C031C99290310B60D5A
:1003000021008C1522000C158529862920008C1DC2
:100310008C290130B7008D29B70122000C119029DA
:10032000912920003708F800F808031D3614B50A93
:100330007A2921008C159C299D2922000C15A029C1
:10034000A1290C11A329A4292000C1203608F800F6
:1003500008002030B3000230B40038217808AC0027
:100360007E30AC058D1FAC178D1A2C140230B300F3
:100370002C08B4000E212030B300B40138217808D5
:10038000AC00F130AC050D1DC8290E30AC04C929F4
:10039000AC15B3012C08B4000E212030B30001309D
:1003A000B40038217808AC00AC120D1BAC1601303B
:1003B000B3002C08B4000E212030B3000630B40086
:1003C00038217808AD002D102030B3000930B4007A
:1003D00038217808AE002E100D1E2D148D1D2E1400
:1003E0000630B3002D08B4000E210930B3002E08EA
:1003F000B4000E2108002030B300B4013821780881
:10040000AC002C10B3012C08B4000E212C14B30145
:100410002C08B4000E2108002F08013C031C1E2AE2
:10042000031D162A2E08003C031C1E2A03102F0C45
:10043000FA002E0CF900FF3CB0004D2A2F08023CB8
:10044000031C3A2A031D282A2E08003C031C3A2AC2
:1004500000302E02B30001302F3BB400340CFA0000
:10046000330CF900FA0CF90C3F30FA057908803C9E
:10047000B0004D2AFE302E02B30001302F3BB400F5
:10048000340CFA00330CF900FA0CF90CFA0CF90CE4
:100490001F30FA057908403CB0003008FF3CB0003E
:1004A0002030B3000330B40038217808B20030089F
:1004B00032020319652A0330B3003008B4000E215C
:1004C0000430B3003008B4000E213008A400080046
:1004D000AD01AC01AE012E080F3C031C9F2A210088
:1004E0009D1420002F1021009D18792A20002F1420
:1004F000210020002F18852A2F1021009D18832A03
:1005000020002F142100792A20000230F70021005A
:100510009D1C8C2AF70B882A1C08FA001B08200057
:10052000B0007A08B1003008F8003108F900790805
:10053000FA007808AC077908AD3DAE0A6B2AAD0C1D
:10054000AC0CAD0CAC0CAD0CAC0CAD0CAC0C0F3061
:10055000AD05230BD82A22082D02031CBD2A031D3A
:10056000B52A2C0821020318BD2A2D08A2002C0848
:10057000A100F8002208F900082B01302C07F80030
:1005800000302D3DFA007A082202031CD72A031DF1
:10059000CD2A210878020318D72A2D08A2002C089A
:1005A000A100A3012108F8002208F900082B042B60
:1005B0002D082202031CEA2A031DE22A21082C022C
:1005C0000318EA2A2D08A2002C08A100F80022082E
:1005D000F900082B01302107AF000030223DB000A8
:1005E0002D02031C042B031DF92A2C082F020318CB
:1005F000042B2D08A2002C08A1000130A300210823
:10060000F8002208F900082B2108F8002208F90058
:100610000800AC018D1B2C148D1AAC140D1B2C156D
:100620000D19AC150D1A2C168D19AC162C082002BC
:100630000319202B2C08A0000130F800232B232BBA
:100640000030F800232B8031822B850184011F307C
:100650008305743021009900FF302000A0002300A2
:100660008C018D01220092019101940193010D10E2
:1006700021000D1002302000AC00FA30BC00032035
:10068000AC0B3D2B182822000C160A302000BC00B1
:1006900003200330B300B4010E210430B300B401D1
:1006A0000E21A921FB21AF01AE010C22682279089D
:1006B000AD007808AC007908AF007808AE000C22D5
:1006C0000B30B300B4010E21A801A701AB0127082C
:1006D000DC3C031D722B2808053C031D722B0130E6
:1006E000AB00752BA70A0319A80AAB080319812BC5
:1006F0008C1F7E2B22000D10802B200022000D1459
:100700002000092BF8080319872BA921FB21A90A2E
:100710000319AA0A8D1F902B22008D149F2B2000F5
:100720000039F7002A080139FA0077087A0403191A
:100730009D2B22008D149F2B200022008D10200065
:1007400068227908AD007808AC007908AF00780815
:08075000AE000C22672B6300D0
:020000040001F9
:04000E00043FFF1E8E
:00000001FF
